:1000000028C04CC061C24AC049C014C247C046C0E3
:1000100045C044C043C042C041C040C03FC00000D2
:10002000000036000000000037000000000038002B
:10003000020202020202020202020102040810206D
:1000400020041008010200000400000000008303E7
:10005000EC0311241FBECFE5D1E0DEBFCDBF10E021
:10006000A0E6B0E0E4E6F8E002C005900D92A23C04
:10007000B107D9F721E0A2ECB0E001C01D92AE3289
:10008000B207E1F710E0C8E2D0E003C02197FE011B
:10009000D3D3C732D107D1F791D2D8C3B1CF089506
:1000A000CF92DF92EF92FF920F931F93CF93DF9344
:1000B0006C017A018B01C0E0D0E0CE15DF0589F03C
:1000C000D8016D918D01D601ED91FC910190F081E7
:1000D000E02DC6010995892B11F47E0102C02196FD
:1000E000ECCFC701DF91CF911F910F91FF90EF905F
:1000F000DF90CF90089590E0FC01EC5BFF4F3491CE
:10010000FC01E65CFF4F2491FC01E05DFF4FE491B0
:10011000EE2339F1332399F0323071F028F4313085
:1001200071F48AB58F770AC0333011F0343039F466
:100130008CB58F7D8CBD03C08AB58F7D8ABDF0E004
:10014000EE0FFF1FE65DFF4FA591B4918FB7F894B6
:10015000EC91611103C020952E2301C02E2B2C930E
:100160008FBF0895CF93DF9390E0FC01E65CFF4FD3
:100170002491FC01E05DFF4F8491882361F190E0C0
:10018000880F991FFC01EC5DFF4FC591D491FC01D4
:10019000E65DFF4FA591B491611109C09FB7F89436
:1001A0008881209582238883EC912E230BC06230B6
:1001B00061F49FB7F8943881822F809583238883D8
:1001C000EC912E2B2C939FBF06C08FB7F894E8813B
:1001D0002E2B28838FBFDF91CF9108953FB7F894DE
:1001E0008091070190910801A0910901B0910A0145
:1001F00022B708B601FE05C02F3F19F00196A11DD8
:10020000B11D3FBFBA2FA92F982F8827820F911DAC
:10021000A11DB11DBC01CD0146E0660F771F881FEF
:10022000991F4A95D1F708958F929F92AF92BF92EE
:10023000CF92DF92EF92FF92D1DF4B015C0180ED14
:10024000C82E87E0D82EE12CF12CC8DFDC01CB01D1
:1002500088199909AA09BB09883E9340A105B105EF
:1002600058F021E0C21AD108E108F10888EE880EA2
:1002700083E0981EA11CB11CC114D104E104F10457
:1002800021F7FF90EF90DF90CF90BF90AF909F90BD
:100290008F90089520910D0130910E012817390794
:1002A00071F490910B0180910C01981741F0E0914D
:1002B0000B01F0E0EE53FF4F808190E008958FEF47
:1002C0009FEF08951F93CF93DF93DC015C962D91F0
:1002D0003C915D972115310539F481E090E013964A
:1002E0009C938E9312973DC05196ED91FC9152973D
:1002F00050969C915097892F80951FB75E964C9190
:100300005E9741FB772770F941FD6095F894408135
:10031000772311F0492B01C048234083E90121973D
:10032000F1F748E0508160FF02C0592B01C058230B
:100330005083E9012197F1F76695415099F77723AA
:1003400021F090818923808303C08081982B908342
:100350001FBF5C968D919C915D970197F1F721E00D
:1003600030E0C901DF91CF911F91089520910D01D7
:1003700030910E012817390769F480910C01209102
:100380000B0190E0805C9F4F821B910960E470E05C
:100390002CD2089580E090E0089520910D013091D5
:1003A0000E0128173907B9F490910B0180910C01C7
:1003B000981789F0E0910B01F0E0EE53FF4F808138
:1003C00020910B0130E02F5F3F4F2F733327209395
:1003D0000B0190E008958FEF9FEF0895E0910D01DC
:1003E000F0910E01E817F90769F4A389B4899C918B
:1003F0008589809589238C9310920E0110920D01AE
:1004000081E0089580E00895089580E090E00895E7
:10041000009761F0FC0101900020E9F73197AF01EE
:10042000481B590BBC018FE091E03ACE80E090E090
:10043000089508D21F920F920FB60F9211242F9396
:100440003F938F939F93AF93BF93809103019091BC
:100450000401A0910501B09106013091020120E351
:10046000230F2D3720F44096A11DB11D05C023EBAD
:10047000230F4196A11DB11D20930201809303011A
:1004800090930401A0930501B093060180910701A8
:1004900090910801A0910901B0910A010196A11D56
:1004A000B11D8093070190930801A0930901B093B7
:1004B0000A01BF91AF919F918F913F912F910F9022
:1004C0000FBE0F901F9018951F920F920FB60F92AC
:1004D00011242F933F934F935F936F937F938F9349
:1004E0009F93AF93BF93EF93FF93E0910D01F09132
:1004F0000E01309709F451C0968DA685B785858584
:1005000091FF04C09C91892329F447C09C918923C1
:1005100009F043C0A389B4899C918589809589237A
:100520008C93868997890197F1F7608D718DA685E7
:10053000B785558538E020E0CB010197F1F7822F90
:1005400090E095958795282F4C91452309F02068D8
:10055000315091F7868D81FD209580910C0190E0BE
:1005600001968F73992730910B01381749F0A091AC
:100570000C01B0E0AE53BF4F2C9380930C0103C02D
:10058000868D8160868F828D938D0197F1F7A38987
:10059000B4899C918589892B8C93FF91EF91BF91B0
:1005A000AF919F918F917F916F915F914F913F910B
:1005B0002F910F900FBE0F901F90189578948AB5C9
:1005C00082608ABD8AB581608ABD83B7826083BF3D
:1005D00083B7816083BF89B7826089BF80B782603B
:1005E00080BF3298319A309A379A8CB580648CBD2E
:1005F00060E081E0B7DD61E080E0B4DD10922A01C7
:1006000010922901109228011092270110922601C0
:100610001092250187E190E090932C0180932B01AB
:1006200040911B01453010F521E0209325011092E7
:10063000260165E170E0709328016093270167E06F
:1006400070E070932A01609329013BB730623BBF91
:1006500065E370E0709323016093220101C0220FD3
:100660004A95EAF7209324010197F1F78091290137
:1006700090912A01892B19F180910D0190910E0121
:1006800021E08F309207D9F0009709F0A7DE809122
:100690002D018E7F80932D0110920C0110920B0181
:1006A0008FE091E090930E0180930D01E091220183
:1006B000F0912301908180912401892B808382E72E
:1006C00090E0A6DE80E890E0A3DE80E990E0A0DE86
:1006D0008EE990E09DDEA8DD8CEA90E099DEA4DD55
:1006E00061E084E03FDD8FE091E040DE892BD9F3CB
:1006F0008FE091E052DE813311F461E001C060E0EF
:1007000084E0F9DCF0CF109212011092110188EE12
:1007100093E0A0E0B0E08093130190931401A093C4
:100720001501B093160184E690E090931001809338
:100730000F011092260110922501109228011092AB
:10074000270110922A011092290110922C01109277
:100750002B0160912D016E7F6D7F60932D01669559
:10076000617081E0682780E0C6DC61E080E0FADC4F
:10077000EAE3F0E0E491E0931F01E0E3F0E0E491CC
:10078000F0E0EE0FFF1FE65DFF4F8591949190938F
:1007900021018093200160E081E0E4DC80912D0163
:1007A00081FD03C061E081E0A6DC81E080931B0154
:1007B000EBE3F0E0E491E0931C01E1E3F0E0E4918D
:1007C000F0E0EE0FFF1FE25EFF4F85919491909352
:1007D0001E0180931D01089584E690E0909310011E
:1007E00080930F018FE091E0F9CD97FB072E16F46F
:1007F000009406D077FD08D00BD007FC05D03EF45E
:10080000909581959F4F0895709561957F4F0895BC
:10081000AA1BBB1B51E107C0AA1FBB1FA617B70726
:1008200010F0A61BB70B881F991F5A95A9F7809542
:100830009095BC01CD010895EE0FFF1F0590F49136
:10084000E02D099481E090E0F89400C010E0C8E247
:10085000D0E003C0FE01F0DF2196C932D107D1F705
:04086000F894FFCF3A
:10086400000000006201500005024F00B601CD01F6
:100874004A010D0A2B5354574D4F443D300D0A0085
:100884000D0A2B53544E413D48432D30350D0A007B
:100894000D0A2B53544F4155543D310D0A000D0A96
:1008A4002B53544155544F3D300D0A00626C75650D
:1008B400746F6F746820636F6E6E65637465642112
:0208C4000A0028
:00000001FF
